:1000000078EF0EF01200FFFF2DEF07F01200FFFF58
:100018006BEF08F01200FFFFFFFFFFFFFFFFFFFF7E
:1008000078EF0EF01200FFFFFFFFFFFFFFFFFFFF7B
:10082A000100081D0000DD000000080000009368B8
:10083A00F26AF16AF06AD09E880ED56E0001606B8A
:10084A00A09AA86B010EA96F606BBD6B090EBD5D06
:10085A003DE2BDC0E6FFCEDAE552E66E110E0001BA
:10086A00BD25EA6A710FE96E000EEA22E552E750E9
:10087A00EF6E110EBD25EA6A710FE96E000EEA22CB
:10088A00EF501F0BE66EBD51EA6AB40FE96E000E17
:10089A00EA22E552E750EF6EBDC0E6FFABDAE55259
:1008AA007F080AE20001BD51EA6AAB0FE96E000E49
:1008BA00EA22010EEF6E08D00001BD51EA6AAB0FC1
:1008CA00E96E000EEA22EF6ABD2BC0D78A0503E162
:1008DA00010EC16F01D0C16B12000001A85101E0E5
:1008EA001AD90001C10501E101D8120038EC0EF055
:1008FA00ECC0C2F009D9040E0001C85D02E2C86B5F
:10090A00DFD038EC0EF0ECC0C3F0FED838EC0EF0B5
:10091A00ECC0C4F0F9D838EC0EF0ECC0C5F0F4D84D
:10092A0038EC0EF0ECC0C6F0EFD80001616B626BD8
:10093A00C76B080EC75D29E2010EC7C0E7FFE75281
:10094A0004E0E846FE0BE706FCE10001C315C7C058
:10095A00E7FFE75204E0E8427F0BE706FCE100010B
:10096A00BE6F070ED880C755026EBE51025204E010
:10097A00E846FE0B0206FCE1006E016A0050000127
:10098A00611301506213C72BD4D7636B646BC76BB7
:10099A00080EC75D29E2010EC7C0E7FFE75204E06F
:1009AA00E846FE0BE706FCE10001C415C7C0E7FFF5
:1009BA00E75204E0E8427F0BE706FCE10001BE6F64
:1009CA00070ED880C755026EBE51025204E0E846AF
:1009DA00FE0B0206FCE1006E016A0050000163137F
:1009EA0001506413C72BD4D7656B666BC76B080EAF
:1009FA00C75D29E2010EC7C0E7FFE75204E0E846F7
:100A0A00FE0BE706FCE10001C515C7C0E7FFE75288
:100A1A0004E0E8427F0BE706FCE10001BE6F070E27
:100A2A00D880C755026EBE51025204E0E846FE0B5A
:100A3A000206FCE1006E016A0050000165130150D4
:100A4A006613C72BD4D7676B686BC76B080EC75D75
:100A5A0029E2010EC7C0E7FFE75204E0E846FE0BB1
:100A6A00E706FCE10001C615C7C0E7FFE75204E04C
:100A7A00E8427F0BE706FCE10001BE6F070ED88053
:100A8A00C755026EBE51025204E0E846FE0B02064A
:100A9A00FCE1006E016A00500001671301506813FF
:100AAA00C72BD4D7C251696F6A6B6B6B6C6B6D6B5A
:100ABA006E6B6F6B706B716B726B010EA86FC86B8C
:100ACA0012000001A56BA66B1D0EA55D000EA659AE
:100ADA0004E2A52B000EA623F7D7BE6BBE6BBE6B36
:100AEA00BE6BBE6B12000001A56BA66B3C0EA55D2A
:100AFA00000EA65904E2A52B000EA623F7D7BE6B5B
:100B0A00BE6BBE6B1200120031EC0EF0E80ED76E0F
:100B1A00900ED66E1200060E0001E55D03E36D50DD
:100B2A00020B01E066D10001BD6B080EBD5D65E2F6
:100B3A00BD51E96EEA6AD890E936EA36950EE92699
:100B4A00000EEA22EE6AED6ABD51EA6AAB0FE96E5F
:100B5A00000EEA22EF504FE0C1512CE1A00E036EC5
:100B6A008C0E046E056ABD51E96EEA6AD890E936C0
:100B7A00EA36610EE926000EEA22EECF06F0EFCF42
:100B8A0007F0086A0650035C006E07500458016EAD
:100B9A0008500558026EBD51E96EEA6AD890E936E6
:100BAA00EA36610EE926000EEA2200C0EEFF01C015
:100BBA00EDFF21D0BD51E96EEA6AD890E936EA36EE
:100BCA00610EE926000EEA22EECF00F0EFCF01F027
:100BDA00000ED8800056010E0156BD51E96EEA6A30
:100BEA00D890E936EA36610EE926000EEA2200C0FC
:100BFA00EEFF01C0EDFFBD2B98D7816BBD6B080ED0
:100C0A00BD5D01E3A5D0BD51EA6AB40FE96E000EDD
:100C1A00EA22EF50000802E3000E01D0010E016E35
:100C2A00BD51EA6AB40FE96E000EEA22EFCF00F076
:100C3A00090E005C02E3000E01D0010E011423E04C
:100C4A00BD51E96EEA6AD890E936EA36610EE926BC
:100C5A00000EEA22EECF00F0EFCF01F0BD51EA6AB2
:100C6A00B40FE96E000EEA22EF04E96EEA6AD89040
:100C7A00E936EA36950EE926000EEA2200C0EEFFB2
:100C8A0001C0EDFF63D0C15131E1BD51EA6AB40F31
:100C9A00E96E000EEA22EF5002E1000E01D0010EC9
:100CAA00006EBD51E96EEA6AD890E936EA36610EFD
:100CBA00E926000EEA22500ED880EE54460EED5474
:100CCA0002E3000E01D0010E00140FE0BD51EA6AE2
:100CDA00B40FE96E000EEA22EF50F70FEA6ADD0F51
:100CEA00E96E000EEA22EF50811330D0BD51EA6A54
:100CFA00B40FE96E000EEA22EF5002E1000E01D0B5
:100D0A00010E006EBD51E96EEA6AD890E936EA36FC
:100D1A00610EE926000EEA22800ED880EE54000EFB
:100D2A00ED5402E3000E01D0010E00140FE0BD5194
:100D3A00EA6AB40FE96E000EEA22EF50F70FEA6A88
:100D4A00DD0FE96E000EEA22EF508113BD2B57D753
:100D5A00BD6B080EBD5D3CE2C15113E1BD51E96EA8
:100D6A00EA6AD890E936EA36950EE926000EEA22B2
:100D7A00EECFC9F0EFCFCAF0500EC95F460ECA5B7C
:100D8A0012D0BD51E96EEA6AD890E936EA36950E74
:100D9A00E926000EEA22EECFC9F0EFCFCAF0800EA4
:100DAA00C95F000ECA5BBD51E824EA6A710FE96E99
:100DBA00000EEA22C9C0EFFFBD51E824010FEA6A1A
:100DCA00710FE96E000EEA22CAC0EFFFBD2BC1D730
:100DDA0004010CBF0BD01A0EE66E710EE66E000E01
:100DEA00E66E0DEC0CF0E552E552E5520001A86BF7
:100DFA00606B1200D9CFE6FFE1CFD9FFFE0EDB50C0
:100E0A00A96EA69EA69CA680A8CFBEF00001BE51E0
:100E1A0000D0E552E7CFD9FF1200D9CFE6FFE1CFE4
:100E2A00D9FFFE0EDB50A96EFD0EDB50A86EA69E02
:100E3A00A69CA684F29E550EA76EAA0EA76EA6823F
:100E4A00A6B2FED7F28EA694E552E7CFD9FF1200DA
:100E5A00DACFE4FFE2CFDAFFE9CFE4FFEACFE4FF3B
:100E6A00F6CFE4FFF7CFE4FFF5CFE4FFF3CFE4FFDB
:100E7A00F4CFE4FFFACFE4FF00EE09F0020EE80433
:100E8A0003E3EECFE4FFFBD700EE00F0090EE8041F
:100E9A0003E3EECFE4FFFBD7E652040108BF7ED09E
:100EAA000A0EE66E8B0EE66E000EE66E47EC0CF04E
:100EBA00E552E552E55231EC0EF0FF0E00018B5D72
:100ECA0010E104010CBF0CD01A0EE66E710EE66E2C
:100EDA00000EE66E0DEC0CF0E552E552E552F1D744
:100EEA005DD0F00E8B5D5AE1BD6B090EBD5D4EE221
:100EFA00BD29EA6A8B0FE96E000EEA22EF50E66E10
:100F0A00110EBD25EA6A710FE96E000EEA22E5525A
:100F1A00E750EF6EBD29EA6A8B0FE96E000EEA22EE
:100F2A00EF50E66EBDC0E6FF78DFE552E552110EDE
:100F3A000001BD25EA6A710FE96E000EEA22EF5040
:100F4A001F0BE66EBD51EA6AB40FE96E000EEA2283
:100F5A00E552E750EF6EBD29EA6A8B0FE96E000E83
:100F6A00EA22EF507F0809E2BD51EA6AAB0FE96E47
:100F7A00000EEA22010EEF6E07D0BD51EA6AAB0FEE
:100F8A00E96E000EEA22EF6ABD2BAFD78A0504E1AB
:100F9A00010EC16FF29602D0C16BF2860001C10543
:100FAA0002E0000E01D0010E0B6EF250040B01E0BC
:100FBA00010E0B1405E0F294A7DD0001C82B62D0E4
:100FCA00C15102E0000E01D0010E0B6EF250040B6B
:100FDA0001E0010E0B140EE0F294605104E18A0E56
:100FEA00D76ED66A4FD0010EA86FA96F8A0ED76E38
:100FFA00D66A48D0C15102E0000E01D0010E0B6E34
:10100A00F250010B0B143EE08150100B01E0010E6F
:10101A00BE6FF29059EC0EF0F3CFA5F0F4CFA6F024
:10102A000001000EA55F8A0EA65BA95107E08A0E91
:10103A00D76ED66AA96BBEC0AAF024D0AA51BE5DEB
:10104A0002E0000E01D0010E0B6EA95102E0000E63
:10105A0001D0010E0B1416E08A0ED76ED66A6051C3
:10106A00E96EEA6AD890E936EA36610EE926000E98
:10107A00EA22A5C0EEFFA6C0EDFF080E605D01E200
:10108A00602B00D0E55200EE08F0090EE80403E3F5
:10109A00E5CFEDFFFBD700EE0AF0020EE80403E30A
:1010AA00E5CFEDFFFBD7E5CFFAFFE5CFF4FFE5CFBC
:1010BA00F3FFE5CFF5FFE5CFF7FFE5CFF6FFE5CF85
:1010CA00EAFFE5CFE9FFE5CFDAFF1100D8CFE4FF69
:1010DA00E0CFE4FFE46EDACFE4FFE2CFDAFFE652D4
:1010EA00E552E5CFDAFFE550E5CFE0FFE5CFD8FFDF
:1010FA00100004011051600BE842E842E842E8425D
:10110A00E842000901E055D01151070A51E00B0AE3
:10111A004FE0070A40E0010A2CE00B0A28E0020A25
:10112A0026E0030A22E0080A12E0010A0EE00F0A8A
:10113A000AE0030A01E03CD00001010ED66F00016B
:10114A00040EE56F36D036D834D090D832D00001AC
:10115A00010ED66F0001E70ED76F000ED86F00019F
:10116A00E6930001010EDB6F24D0A8D822D0F4D870
:10117A0020D00001010ED66F040114510001D76F6F
:10118A00D86BE80ED727000ED8230001E69300019A
:10119A00010EDB6F0ED00001010ED66F040114514F
:1011AA00EA6AE80FE96E000EEA2212C4EFFF01D0E4
:1011BA0000D01200800E0401105D57E11351030A9A
:1011CA0034E0010A10E0030A01E04DD00001010EEB
:1011DA00D66F0001960ED76F1A0ED86F120E000145
:1011EA00DB6FDC6B40D00001010ED66F0401125197
:1011FA00F66EF76AD890F636F736600EF6261B0EAC
:10120A00F7220900F5CFD7F00A00F5CFD8F0020E81
:10121A000001F76AD725F66ED851F7220900F5CFF3
:10122A00DBF00A00F5CFDCF01ED00001010ED66F0C
:10123A0004011251F66EF76AD890F636F736640E44
:10124A00F6261B0EF7220900F5CFD7F00A00F5CFD4
:10125A00D8F0D7C0F6FFD8C0F7FF0800F550000154
:10126A00DB6FDC6B00D00001E68312000001010E87
:10127A00D66F0F0EE66E710EE66E0F0EE66E36EC48
:10128A000DF0E552E552E552010EE66EE80EE66E05
:10129A00000EE66E36EC0DF0E552E552E55212C448
:1012AA00E7F00401125104E10001050EE56F05D0D3
:1012BA000001060EE56FF8EC0BF012000401186B42
:1012CA00196B040110511F0B020A14E0030A0EE005
:1012DA00010A01E033D00001010ED66F0401188122
:1012EA000001E6A102D00401188328D00001010EF2
:1012FA00D66F24D00001010ED66F040114510F0BD2
:10130A00080DF350016A000F006E040E01221451F9
:10131A00800B01E0010E040DF35000010024D96F87
:10132A00000E0120DA6FD9C0E9FFDAC0EAFFEF50F8
:10133A00040B03E00401010E186F00D00001D6056A
:10134A000AE10001180ED76F040ED86F0001E69368
:10135A000001020EDB6F12000401120510E11051A8
:10136A001F0B00090CE10001010ED66F030E0401E8
:10137A00115D03E10001E68102D00001E69104015A
:10138A0012513AE110511F0B020836E114510F0BAA
:10139A00000932E00001010ED66F040114510F0B4F
:1013AA00080DF350016A000F006E040E0122145159
:1013BA00800B01E0010E040DF35000010024D96FE7
:1013CA00000E0120DA6F030E0401115D07E1840E9D
:1013DA00D9C0E9FFDAC0EAFFEF6E0ED014AF06D02B
:1013EA00D9C0E9FFDAC0EAFFEF6A06D0880ED9C091
:1013FA00E9FFDAC0EAFFEF6E12006C500BE104015C
:10140A0000513C0BE842E8420D0802E108D801D03D
:10141A003CD804D0040E6C5C01E147D81200D9CF45
:10142A00E6FFE1CFD9FFE6520001D56BD66BDB6B45
:10143A00DC6B7EEC08F0DF6ADF50006E016A010E99
:10144A00005C000E01581BE20001D65101E017D0E2
:10145A00F76ADF34FE0BF736F66E6A0EF6261B0EB7
:10146A00F7220900F5CF00F00800F5CF01F004D00B
:10147A0001C0FAFF0050F96EFBDFDF2ADDD7DDD8A5
:10148A00E552E552E7CFD9FF1200020E0001D55D01
:10149A000AE196D8040100BD03D0C80E006F02D03D
:1014AA00880E006F01D00FD91200040E0001E55D0D
:1014BA000AE112C46EFF6E50000803E2050EE56FE2
:1014CA0002D0030EE56F0001D5050AE10BD804012D
:1014DA0004BD03D0C80E046F02D0880E046F01D079
:1014EA00F2D81200D9CFE6FFE1CFD9FF020EE126EA
:1014FA000001080EDB5D000EDC5905E2DBC0DEFFF1
:10150A00DCC0DDFF03D0080EDE6EDD6A0401049341
:10151A000491010EDB500413DFCF05F4000EDB50FB
:10152A000001DB5F010EDB50DC5B180ED96F040E85
:10153A00DA6F0001E6A31ED0D9CFE9FFDACFEAFFBE
:10154A00EE50ED1016E0D7C0F6FFD8C0F7FF08003E
:10155A00F550D9C0E9FFDAC0EAFFEF6E0001D92BD6
:10156A00000EDA23D72BD823DF06010E01E2DB06B1
:10157A00E3D71CD0D9CFE9FFDACFEAFFEE50ED105E
:10158A0015E0D7C0E9FFD8C0EAFFEF50D9C0E9FF9C
:10159A00DAC0EAFFEF6E0001D92B000EDA23D72B4F
:1015AA00D823DF06010E01E2DB06E4D7020EE15C76
:1015BA0002E2E16AE552E16EE552E7CFD9FF120095
:1015CA00D9CFE6FFE1CFD9FF020EE126030E0401CF
:1015DA000015E76E010EE7CFDBFF01C4DFFFDE5027
:1015EA000001DB27DD50DC23180ED76F040ED86FFD
:1015FA00D9CFE9FFDACFEAFFEE50ED1014E0D7C0F9
:10160A00E9FFD8C0EAFFEF50D9C0E9FFDAC0EAFF24
:10161A00EF6ED92B000EDA23D72BD823DF06010E63
:10162A0001E2DB06E5D7020EE15C02E2E16AE5527D
:10163A00E16EE552E7CFD9FF12000001D6510CE165
:10164A000401080E016F100E026F040E036F840E60
:10165A00006F0401046F35D0040110AF22D00001DD
:10166A00DB510401165D0001DC510401175904E243
:10167A0016C4DBF017C4DCF035DF0001010ED56FAC
:10168A000401080E016F100E026F040E036F800E24
:10169A00006F0401180E066F040E076FC80E046F60
:1016AA0010D00001020ED56F0401056BC80E046F3D
:1016BA000401080E016F180E026F040E036FC80EA4
:1016CA00006F6D9812000001D56B0401080E016FBE
:1016DA00100E026F040E036F880E006F0401046B74
:1016EA001200040110511F0B010801E079D01451B6
:1016FA0001E076D0060E115D2EE11351230A28E08F
:10170A00010A13E0030A01E024D00001020ED66F99
:10171A000001E70505E10001BA0ED76F1A0ED86F6E
:10172A00090E0001DB6FDC6B14D00001020ED66FCC
:10173A000001E70505E10001110ED76F1B0ED86FF6
:10174A000001E70504E14F0E0001DB6FDC6B01D0FD
:10175A0000D00001E68304011051600BE842E84220
:10176A00E842E842E842010801E03AD011510B0A86
:10177A0031E0080A21E0090A19E0080A09E00B0A1F
:10178A0005E0080A01E02CD02CD82AD02BD828D082
:10179A000001020ED66F0001E90ED76F000ED86F56
:1017AA000001E6930001010EDB6F1AD00001020E60
:1017BA00D66F13C4E9F014D00001020ED66F0001EF
:1017CA00EA0ED76F000ED86F0001E6930001010EF2
:1017DA00DB6F06D00001020ED66F12C4EAF000D009
:1017EA001200120012000001EB6B1E0E716E040152
:1017FA000A0E096F200E0A6F040E0B6F880E086F0F
:10180A0004012A0E0E6F040E0F6F400E0C6F1200A9
:10181A00D9CFE6FFE1CFD9FFE652FC0EDB501A081A
:10182A0005E21A0EF36EFC0EF3CFDBFFDF6AFC0E45
:10183A00DB50DF5C19E2DF50E76EFD0EDBCFE9FF1C
:10184A00FE0EDBCFEAFFE750E926000EEA22EF5050
:10185A00E66EDF50EA6A2A0FE96E040EEA22E552C2
:10186A00E750EF6EDF2AE3D7FC0EDBCF0DF4400E14
:10187A0004010C170C7D880E0C13E552E552E7CFD4
:10188A00D9FF1200D9CFE6FFE1CFD9FF0001EB6BF8
:10189A00040108BF31D0FC0EDBCF00F00951D8801B
:1018AA00005403E2FC0E09C4DBFF0001EB6BFC0EE3
:1018BA00DB50EB5D19E2EB51EA6A200FE96E040E88
:1018CA00EA22EF50E66EEB51E76EFD0EDBCFE9FF41
:1018DA00FE0EDBCFEAFFE750E926000EEA22E552C8
:1018EA00E750EF6EEB2BE3D704010A0E096F400EA7
:1018FA000817087D880E08130001EB5100D0E55245
:10190A00E7CFD9FF12006DA60FD802D06DB613D853
:10191A000001E50508E16DBA06D0686A696A69805E
:10192A006988020EE56F12006D6A696A6D860001A8
:10193A00010EE56F12006D6A696A0001E56B12001B
:10194A00A0EF0CF00001E55101E13AD06850040B18
:10195A0004E06950040B01E041D86DB231D06850FF
:10196A00010B04E06950010B01E059D86850100BD3
:10197A0004E06950100B01E024D86850400B04E0E1
:10198A006950400B01E040D86850200B04E06950D0
:10199A00200B01E03BD86850020B04E06950020BAF
:1019AA0001E03BD8030E0001E55D01E209D0685071
:1019BA00080B06E06950080B03E002EC0AF068968F
:1019CA001200698468986D82A19AF290A08AF286C0
:1019DA000300F2B007D8A09AF29612006D926994A9
:1019EA00689412000001E6A10ED0F8DF6D840001B0
:1019FA00080EEE6F070EEF6FEE07000EEF5BEE516B
:101A0A00EF11FAE16D941200689C120070A003D0E5
:101A1A0068EC0BF07090689A1200689212006A6A79
:101A2A00686A9F0E6B6E7B0E696E6E6A0F0EE66EAB
:101A3A00710EE66E0F0EE66E14D8E552E552E552C7
:101A4A00160E706E68A602D06896FCD76D9868EC80
:101A5A000BF00001E6910001E76B0001030EE56F50
:101A6A001200D9CFE6FFE1CFD9FFFD0EDBCFE9FFA8
:101A7A00FE0EDBCFEAFFFC0EDB5004E0EE6AFC0E42
:101A8A00DB06F9D7E552E7CFD9FF120012010002AF
:101A9A0000000008D804716901000102000109026E
:101AAA00290001010080320904000002030000003D
:101ABA00092101010001224F00070581031A000ACA
:101ACA00070501030A000A0403090410035200432C
:101ADA00002D0045004C00450043002C03520043F2
:101AEA00002D00550053004200200049006E00748A
:101AFA000065007200660061006300650020005600
:101B0A000032002E00310005010904A1010901A1DA
:101B1A000005010930093109320933093409350947
:101B2A00360937150026007F9508751081020509C8
:101B3A001901290895087501810205010900158016
:101B4A00257F95097508810209001580257F950A68
:101B5A0075089102C0C0A81AA81AD11AD51AE51A8E
:101B6A00EC162A0EF66E080EF76E000EF86E0001DD
:101B7A000900F550D06F0900F550D16F03E1D06725
:101B8A0001D03DD00900F550CB6F0900F550CC6F5C
:101B9A000900F550CD6F09000900F550E96E0900FA
:101BAA00F550EA6E090009000900F550CE6F0900E8
:101BBA00F550CF6F09000900F6CFD2F0F7CFD3F076
:101BCA00F8CFD4F0CBC0F6FFCCC0F7FFCDC0F8FFFA
:101BDA000001CE5302E1CF5307E00900F550EE6E43
:101BEA00CE07F8E2CF07F9D7D2C0F6FFD3C0F7FF86
:101BFA00D4C0F8FF0001D007000ED15BBFD7120096
:101C0A00929894901CEC04F01CD8060E0001E55D35
:101C1A0002E222D8FAD7F294F2908A0ED76ED66AE6
:101C2A000001C10504E1E80ED76E900ED66EF28E61
:101C3A00F28AC15101E1F2860FD872EC04F0FCD7A6
:101C4A0012000F0EC112140E6F6E0001E56B000137
:101C5A00E66B0001E76B120088EC0CF06FBE02D055
:101C6A00A7EC0CF012000001080EED6F0F0181B80D
:101C7A003CEF0EF066EC05F00F0181B83CEF0EF078
:101C8A0078EC05F00F0181A8D89081B8D8800001BE
:101C9A00EC33ED2F45EF0EF078EC05F066EC05F02D
:101CAA0000000001EC511200D9CFE6FFDACFE6FFBF
:101CBA00E1CFD9FFE2CFDAFFE652E652D650DF6E25
:101CCA00010ED7CFDBFFDECF00F0DDCF01F000C081
:101CDA00F3FF01C0F4FFE552E552E552E5CFDAFF22
:101CEA00E7CFD9FF120013EE00F023EE00F0F86AF6
:101CFA000A9CB6EC0DF005EC0EF0FDD712000102BD
:101D0A00040810204080FFFFFFFFFFFFFFFFFFFFD7
:020000040020DA
:020000040030CA
:0E000000240E391E000181000FC00FE00F40DA
:0200000400F00A
:1000000001000200060007000400050009000A00C4
:100010000000FF00FF00FF00FF00FF00FF00FF00E7
:00000001FF
